:1000000035C34FC34EC34DC34CC34BC34AC349C38F
:1000100048C347C346C345C344C343C342C341C3A4
:1000200040C33FC33EC3D4CBD8CBDACBE8CB10CC54
:1000300012CC1CCCC2CB000000000000000000006D
:1000400000000000000000183C3C3C181800181884
:10005000000000666666240000000000000000004A
:100060000000006C6CFE6C6C6CFE6C6C0000001888
:10007000187CC6C2C07C0686C67C1818000000002A
:1000800000C2C60C183066C60000000000386C6C58
:100090003876DCCCCC760000001818183000000050
:1000A0000000000000000000000C1830303030303C
:1000B000180C000000000030180C0C0C0C0C183050
:1000C00000000000000000663CFF3C6600000000ED
:1000D000000000000018187E181800000000000042
:1000E0000000000000000018181830000000000098
:1000F000000000FE00000000000000000000000002
:10010000000000001818000000000002060C183063
:1001100060C080000000000000386CC6C6D6C6C6AD
:100120006C38000000000018387818181818187E6D
:1001300000000000007CC6060C183060C6FE0000FF
:100140000000007CC606063C0606C67C00000000D7
:10015000000C1C3C6CCCFE0C0C1E0000000000FED1
:10016000C0C0C0FC0606C67C00000000003860C0AD
:10017000C0FCC6C6C67C0000000000FEC6060C1807
:100180003030303000000000007CC6C6C67CC6C6D9
:10019000C67C00000000007CC6C6C67E06060C7841
:1001A00000000000000018180000001818000000EF
:1001B00000000000181800000018183000000000AF
:1001C000000C183060C06030180C00000000000007
:1001D00000007E00007E000000000000006030187B
:1001E0000C060C18306000000000007CC6C60C181D
:1001F0001800181800000000007CC6C6DEDEDEDC39
:10020000C07C000000000010386CC6C6FEC6C6C622
:100210000000000000FC6666667C666666FC000006
:100220000000003C66C2C0C0C0C2663C00000000C6
:1002300000F86C66666666666CF80000000000FEFA
:1002400066626878686266FE0000000000FE666212
:100250006878686060F000000000003C66C2C0C0C2
:10026000DEC6663A0000000000C6C6C6C6FEC6C6A8
:10027000C6C600000000003C181818181818183CD2
:1002800000000000001E0C0C0C0C0CCCCC78000004
:10029000000000E6666C6C786C6C66E6000000009E
:1002A00000F060606060606266FE0000000000C6F2
:1002B000EEFED6C6C6C6C6C60000000000C6E6F6FC
:1002C000FEDECEC6C6C600000000007CC6C6C6C69E
:1002D000C6C6C67C0000000000FC6666667C6060E6
:1002E00060F000000000007CC6C6C6C6C6D6DE7C34
:1002F0000E00000000FC6666667C6C6666E6000028
:100300000000007CC6C660380CC6C67C0000000039
:10031000007E7E5A18181818183C0000000000C60D
:10032000C6C6C6C6C6C6C67C0000000000C6C6C695
:10033000C6C6C66C38100000000000C6C6C6C6D6C9
:10034000D6FE6C6C0000000000C6C6C67C387CC6B9
:10035000C6C60000000000666666663C1818183CB9
:100360000000000000FEC68C183060C2C6FE00000F
:100370000000003C303030303030303C00000000B5
:100380000080C0E070381C0E060200000000003C37
:100390000C0C0C0C0C0C0C3C000010386CC6000053
:1003A000000000000000000000000000000000004D
:1003B0000000000000FF0030180C000000000000EA
:1003C00000000000000000000000780C7CCCCC761F
:1003D0000000000000E06060786C6666667C0000EB
:1003E0000000000000007CC6C0C0C67C0000000009
:1003F000001C0C0C3C6CCCCCCC7600000000000047
:1004000000007CC6FEC0C67C00000000001C363226
:10041000307C30303078000000000000000076CCE6
:10042000CCCC7C0CCC78000000E060606C7666661A
:1004300066E6000000000018180038181818183C6C
:1004400000000000000606000E0606060666663C72
:10045000000000E06060666C786C66E600000000FA
:100460000038181818181818183C00000000000070
:100470000000ECFED6D6D6D600000000000000003A
:10048000DC666666666600000000000000007CC650
:10049000C6C6C67C0000000000000000DC66666680
:1004A0007C6060F000000000000076CCCCCC7C0CBE
:1004B0000C1E000000000000DC76666060F00000AA
:1004C0000000000000007CC6701CC67C000000001C
:1004D00000103030FC303030361C000000000000CE
:1004E0000000CCCCCCCCCC7600000000000000009A
:1004F000C6C6C66C38100000000000000000C6C66A
:10050000D6D6FE6C0000000000000000C66C383833
:100510006CC60000000000000000C6C6C6C67E060D
:100520000C78000000000000FECC183066FE0000D1
:100530000000000E181818701818180E000000009F
:100540000018181818181818181800000000007063
:100550001818180E1818187000000076DC0000003B
:100560000000000000000000000000000010386CD7
:10057000C6C6FE000000FDFDFDFDEF00EE041B04FD
:10058000FEFEFEFEEF904A047F3FEE044306EF902E
:10059000098308000BAF0A00050006000700EF0002
:1005A000EE0CEF900080EFB04902EF007F01E18197
:1005B000E202E276E18380014D61747468696173DF
:1005C00020426F64650000000000000064696769F4
:1005D00074616C6572000000000000000000000003
:1005E00042696C6465727261686D656E000000003E
:1005F000000000005665722E20302E3100000000F1
:10060000000000000000000028432932303037008D
:100610000000000000000000000000004B65696E53
:10062000652053442D4B6172746521000000000069
:100630004B65696E652053442D4B617274652121B1
:10064000000000004B65696E65202E626D702D44C0
:1006500061746569656E2100756E62656B616E6EB1
:10066000746572204665686C6572210011241FBE96
:10067000CFE5D4E0DEBFCDBF10E0A0E6B0E0E6E31A
:10068000FDE102C005900D92A037B107D9F712E045
:10069000A0E7B0E001C01D92A43FB107E1F77ED80A
:1006A00049CBAECC0F931F938C01812F99273ED25B
:1006B000802F3CD21F910F91089590917700E92FE0
:1006C000FF27E858FF4F80839F5F90937700933018
:1006D00078F1409179002091780050917A00109241
:1006E000770080917B0090917C00019690937C0034
:1006F00080937B000197805C9A45D4F4842F9927DE
:10070000887F9070982F882733272C7F307063E084
:10071000220F331F6A95E1F7820F931F252F33278E
:1007200043E0369527954A95E1F7820F931FBADF8C
:1007300008950F931F938C01892F992708D2802F3A
:1007400006D21F910F9108958F929F92AF92BF9200
:10075000CF92DF92EF92FF920F931F93CF93DF938D
:10076000D82E062FE42EF22E80E99FEEE2DF84E001
:1007700095E0DFDF1127C8018050984FDADFCD2DDB
:10078000DD27CE018050964FD4DFCF2CDD24C7FC6F
:10079000D0949601220F331FC901B3E0880F991F2F
:1007A000BA95E1F7821B930B0150174F800F911FF1
:1007B000C0DFC601A3E0880F991FAA95E1F7C150D9
:1007C000D54F8C0F9D1FB5DF8EE09E2D98028001C6
:1007D00011240C571140992401501040F8018490C5
:1007E000AA24BB2428C0F694882D8F2119F4C0E0D8
:1007F000D0E014C0C0E0D0E005C0809170009091BE
:10080000710050DF8C2F992721968C159D05ACF334
:100810000BC0809166009091670044DF8C2F992770
:1008200021968C159D05ACF3E394F8E0EF16D9F60C
:100830000894A11CB11C8A2D99278C159D0524F4C0
:10084000EE24F0E8FF2ED0CF93948EE0981609F0B6
:10085000C3CFDF91CF911F910F91FF90EF90DF9069
:10086000CF90BF90AF909F908F900895EF92FF929E
:100870000F931F93CF93DF93E82E062FF42E80E97A
:100880009FEE57DF84E095E054DF1127C8018050C8
:10089000984F4FDFCE2DDD27CE018050964F49DF98
:1008A000C801835F964F45DFCE01895F944F41DFDA
:1008B0008EE09F2D9802E0011124CC57D140FF24F7
:1008C0002197FE01E49010E000E88E2D802329F0AE
:1008D000809170009091710004C0809166009091A9
:1008E0006700E0DE1F5F183011F00695EECFF3943D
:1008F000FEE0FF1629F7DF91CF911F910F91FF9036
:10090000EF9008950F931F93CF93DF93082FEB0180
:10091000CB01B7D9873108F086E18695880F880F1B
:10092000880F18E5181B05C02196602F812F9EDFC8
:10093000185F48814423C1F7DF91CF911F910F9138
:1009400008950F931F93CF93DF93082FEB01CB01F3
:10095000A4D9873108F086E18695880F880F880F23
:1009600018E5181BFE0121964491442329F0602FBD
:10097000812F7CDF185FF6CFDF91CF911F910F9110
:1009800008950F931F93CF93DF938C0180E99FEE1F
:10099000D0DE84E095E0CDDE80E098E0CADE80E045
:1009A0009AE0C7DE83E899E0C4DE8FEA9BE0C1DE0F
:1009B000C0E0D0E0C80176DE21968AE5C03CD807C9
:1009C000C9F7DF91CF911F910F910895CF92DF92D8
:1009D000FF920F931F93CF93DF93CDB7DEB7269788
:1009E0000FB6F894DEBF0FBECDBF6C010091700052
:1009F00010917100DE011196E0E6F0E086E00190D2
:100A00000D928150E1F78091660090916700B9DF07
:100A1000809168009091690080959095909369000D
:100A200080936800909371008093700024E041E20D
:100A30006DE288E489DE109371000093700090E30A
:100A4000F92E00E010E006C022E064E68F2D7CDE87
:100A500080E1F80EFE013196E00FF11D40810F5F3D
:100A60001F4F442389F7B60189E16BDF26960FB645
:100A7000F894DEBF0FBECDBFDF91CF911F910F91D4
:100A8000FF90DF90CF9008951092770010927C0035
:100A900010927B0080E99FEE4CDE84E095E049DE19
:100AA00080E098E046DE80E09AE043DE83E899E06B
:100AB00040DE8FEA9BE03DDE08951F93CF93DF93E6
:100AC00099D083E698EF90936700809366008FE05B
:100AD00090E0909371008093700083E698EF51DF6F
:100AE000C8EBD5E014E6BE01812F2BDF14516496CC
:100AF0001123C9F788E893E118D01092770080E9B4
:100B00009FEE17DE84E095E014DE80E098E011DED1
:100B100080E09AE00EDE83E899E00BDE8FEA9BE04E
:100B200008DEDF91CF911F910895089592989098D3
:100B300090E087FF02C0939A01C09398959A959888
:100B40009F5F983011F0880FF4CF929A0895929891
:100B5000909A90E087FF02C0939A01C09398959A6B
:100B600095989F5F983011F0880FF4CF929A08956E
:100B7000CF93DF938FEEEBDF80E9E9DF85E0E7DFFE
:100B800080E0E5DF86E0E3DF80E0E1DF87E0DFDFD4
:100B900080E0DDDFC0E0D0E08FEFC8DF8FEFC6DFA1
:100BA00021968AE5C03CD807B9F7DF91CF91089527
:100BB0001F93CF93DF93EC01162F05C0FE01219602
:100BC000E4918E2FC4DF1150C8F7DF91CF911F91B0
:100BD00008959198899A8B9A929A8A9A95988D9A63
:100BE000909A889A82E390E0A0DF919A82E390E065
:100BF0009CDF0895929A8A9AECDF68E186E795E097
:100C0000D7DF87E090E091DF68E28EE895E0D0DF03
:100C100082E390E08ADF62E086EB95E0C9DF92989C
:100C20008FEE95DF80E993DF80E091DF80E08FDF5A
:100C30000895BF92CF92DF92EF92FF920F931F938E
:100C4000E0917D00F0917E0060E070E080E090E057
:100C50000995882311F5E0919700F0919800E250F2
:100C6000FE4F8081EE5FF140853509F089C0E1508B
:100C7000FE4F8081EF5FF1408A3A09F081C0EA536C
:100C8000FE4F0081602F772788279927E0917D000C
:100C9000F0917E000995882311F0992773C0E091A7
:100CA0009700F0919800B584C784DD24A0896485FD
:100CB0007727762F66278385680F711D478955270B
:100CC000542F44278689480F511D82899927982FD0
:100CD00088272189820F911DDC2CCC242685200FAA
:100CE000312D311DC20ED31EEE24FF24C0928B0085
:100CF000D0928C00E0928D00F0928E00BB27A49FD2
:100D00008001A59F100DB49F100D112422273327B9
:100D10000C0D1D1D2E1D3F1D00939D0010939E0068
:100D200020939F003093A00045E0880F991F4A95BB
:100D3000E1F7860F971F0197E9D788279927600F5A
:100D4000711F821F931F60938F0070939000809398
:100D5000910090939200B0928000009387001093CE
:100D600088002093890030938A00009399001093A3
:100D70009A0020939B0030939C0080E090E002C09A
:100D80008AE190E01F910F91FF90EF90DF90CF905C
:100D9000BF900895CF93DF93EC0160919D00709117
:100DA0009E0080919F009091A000E0917D00F091C5
:100DB0007E000995882311F0992728C0E0919700BB
:100DC000F091980040E050E083858830B1F420E055
:100DD00030E0DE01E0919700F0919800E40FF51FFC
:100DE000E20FF31F80818D932F5F3F4F2B30310532
:100DF00089F71B8680E090E009C0405E5F4FB096A7
:100E000082E04030580701F781E090E0DF91CF9118
:100E100008951F93142F625070408040904020919D
:100E2000800033274427552752D720918F003091D7
:100E300090004091910050919200620F731F841FA7
:100E4000951F610F711D811D911DE0917D00F09135
:100E50007E00099599271F910895AF92BF92CF9276
:100E6000DF92EF92FF920F931F937B018C0161152C
:100E700071058105910529F462E0E62EF12C012D22
:100E8000112DAF2CB02EC12EDD2460918B007091FE
:100E90008C0080918D0090918E006A0D7B1D8C1DC1
:100EA0009D1DE0917D00F0917E000995882329F039
:100EB00020E030E040E050E02BC0E0919700F0915E
:100EC0009800BC2DAB2D9A2D8827E81AF90A0A0B39
:100ED0001B0BEE0CFF1C001F111FEE0DFF1D81816F
:100EE0009927AA27BB272227382F492F5A2F8081DD
:100EF000280F311D411D511D2F3F8FEF380780E016
:100F0000480780E0580721F42FEF3FEF4FEF5FEFE6
:100F1000CA01B9011F910F91FF90EF90DF90CF9020
:100F2000BF90AF900895FC0191912AE090FF02C01C
:100F300080E801C080E09695980F8191980F21502C
:100F4000A9F7892F992708958F929F92AF92BF9208
:100F5000CF92DF92EF92FF920F931F93CF93DF9385
:100F60007B018C015B016C01A4E0D694C794B7941B
:100F7000A794AA95D1F72A0D3B1D4C1D5D1DE0914C
:100F80007D00F0917E00CA01B9010995882309F01E
:100F900087C1FFE08F2E8E20282D3327E5E0220F1A
:100FA000331FEA95E1F7E0919700F0919800E20F86
:100FB000F31F8081882339F4F0928500E092840049
:100FC00082E090E074C1853E09F46FC18E3219F45D
:100FD00089E590E06CC19385903219F0903109F069
:100FE00064C140E050E0E0919500F0919600E40F7C
:100FF000F51FA0919700B0919800A20FB31FA40F06
:10100000B51F8C9180834F5F5F4F4C30510559F76E
:10101000E0919500F09196008FE28387E091950032
:10102000F0919600903279F58EE28087A09195003C
:10103000B0919600E0919700F0919800E20FF31FB5
:101040008085ED018987A0919500B0919600E0918F
:101050009700F0919800E20FF31F8185FD018287D0
:10106000A0919500B0919600E0919700F0919800C2
:10107000E20FF31F8285ED018B87E0919500F091DF
:101080009600148603C01486903181F0E09195009B
:10109000F09196008185823409F007C182858D34F4
:1010A00009F003C18385803509F0FFC0A091950048
:1010B000B0919600E0919700F0919800E20FF31F35
:1010C0008589FD018587A0919500B0919600E091FA
:1010D0009700F0919800E20FF31F8489ED018E874D
:1010E000A0919500B0919600E0919700F091980042
:1010F000E20FF31F838DFD018787A0919500B091CA
:101100009600E0919700F0919800E20FF31F828D16
:10111000ED01888BA0919500B0919600E091970029
:10112000F0919800E20FF31F878DFD01818BA09154
:101130009500B0919600E0919700F0919800E20F31
:10114000F31F868DED018A8BA0919500B0919600DA
:10115000E0919700F0919800E20FF31F858DFD015B
:10116000838BA0919500B0919600E0919700F0914B
:101170009800E20FF31F848DED018C8B8091970016
:1011800090919800820F931FCEDE982E482D8601F5
:101190007501442311F0415020C0E114F104010510
:1011A000110509F463C00894E108F1080109110967
:1011B00060919D0070919E0080919F009091A00091
:1011C0006E0D7F1D801F911FE0917D00F0917E00CC
:1011D0000995882309F04AC04FE0842F992775E0CC
:1011E000880F991F7A95E1F7A0919700B091980028
:1011F000A80FB91FFD0183858F30C1F5858589153D
:10120000A9F58C9199278F7390702DE030E0BC0187
:10121000629FC001639F900D729F900D11248D50AD
:10122000863100F5E82FFF27EF55FF4F1586ED01BA
:101230008E8D84878C8D8387888D82878E89818728
:101240008C8980878A898783888986838E85858330
:10125000898584838F8183838D8182838B81818340
:10126000898180838C918F3308F493CFEA14FB0437
:101270000C051D05B9F080919D0090919E00A091F4
:101280009F00B091A000A80EB91ECA1EDB1EE091FF
:101290007D00F0917E00C601B5010995882311F00B
:1012A000992705C080E090E002C087E590E0DF91DB
:1012B000CF911F910F91FF90EF90DF90CF90BF9053
:1012C000AF909F908F9008956F927F928F929F9290
:1012D000AF92BF92CF92DF92EF92FF920F931F9344
:1012E000CF93DF937B018C0139014A018091840007
:1012F00090918500AA27BB27E816F9060A071B0765
:1013000020F50894E11CF11C011D111DC0E0D0E086
:10131000570168010894A11CB11CC11CD11CA40177
:101320009301C801B70110DE882319F4C801B70181
:1013300010C0893551F0823041F0219683E0CF3FD3
:10134000D80719F086017501E3CF60E070E080E016
:1013500090E0DF91CF911F910F91FF90EF90DF9080
:10136000CF90BF90AF909F908F907F906F90089597
:1013700020919D0030919E0040919F005091A000CF
:10138000E3DD992708959F92AF92BF92CF92DF92AB
:10139000EF92FF920F931F935B016C019B01AC01D5
:1013A00060E070E080E090E08FDF709394006093E5
:1013B00093007B010027112799242FEF3FEF4FEF78
:1013C0005FEF0AC09394A6019501C801B7017CDFC5
:1013D000A80197017B018C01E114F10401051105BD
:1013E00089F730938500209384009920C1F0809183
:1013F000870090918800A0918900B0918A00809325
:10140000990090939A00A0939B00B0939C00A092A7
:101410008700B0928800C0928900D0928A00892DFE
:1014200099271F910F91FF90EF90DF90CF90BF9081
:10143000AF909F90089509C020E030E000002F5F3A
:101440003F4F45E02D323407C9F701972FEF8F3F0B
:10145000920791F708951F938091CD00882309F496
:101460008EC080916A0090916B00805092400CF485
:101470007BC08091C9009091CA00A091CB00B0912F
:10148000CC000196A11DB11D8093C9009093CA00A4
:10149000A093CB00B093CC002091C5003091C60042
:1014A0004091C7005091C800281739074A075B07C9
:1014B00008F465C020917600332727FD3095809190
:1014C000800099270197821793079CF41092760069
:1014D0006091CF007091D0008091D1009091D200A6
:1014E000BCDC6093CF007093D0008093D1009093C8
:1014F000D2008091CF009091D000A091D100B09106
:10150000D2008F5F9F4FAF4FBF4F11F010E005C06B
:101510001092CD007DD333C07BD36091CF0070910A
:10152000D0008091D1009091D2004091760071DC82
:10153000882311F0115081F710926B0010926A000D
:10154000809176008F5F809376000EC0E0919700C7
:10155000F0919800E20FF31F80812F5F3F4F30938F
:101560006B0020936A00A9D820916A0030916B002B
:1015700082E02030380754F381E090E002C080E040
:1015800090E01F910895209187003091880040914C
:10159000890050918A00609172007091730080916F
:1015A000740090917500D0DC882309F099C0809177
:1015B0007F00803109F494C08091A100882319F044
:1015C00061EA70E004C0609195007091960084E635
:1015D00099D95ADAE0919500F091960065857727C0
:1015E00088279927982F872F762F66276093CF001B
:1015F0007093D0008093D1009093D2002685620F23
:10160000711D811D911D982F872F762F662760935E
:10161000CF007093D0008093D1009093D2002785A3
:10162000620F711D811D911D982F872F762F6627C0
:101630006093CF007093D0008093D1009093D2003C
:101640002089620F711D811D911D6093CF007093E1
:10165000D0008093D1009093D20021893327442772
:101660005527542F432F322F22272093C500309324
:10167000C6004093C7005093C800A2892A0F311DAD
:10168000411D511D542F432F322F22272093C50077
:101690003093C6004093C7005093C800E3892E0FD3
:1016A000311D411D511D2093C5003093C60040934C
:1016B000C7005093C8001092760024E230E03093C7
:1016C0006B0020936A0040E0A4DB81E08093CD00B2
:1016D0001092C9001092CA001092CB001092CC0058
:1016E000089510927200109273001092740010927C
:1016F000750010929400109293008FEF9FEF9093DB
:1017000085008093840084D2882311F0992708955E
:1017100090DA882319F480E090E0089599270895DD
:101720001F9331DE182F8091930090919400AA2787
:10173000BB278093720090937300A0937400B093C2
:10174000750021DF88DE812F99271F91089580E899
:1017500088B916B89FD084ED90E09093980080935C
:10176000970084ED92E0909396008093950082E438
:101770009DE090937E0080937D0084EC9DE09093AB
:101780008300809382008FEF9FEF9093850080937A
:101790008400109294001092930008950F931F9369
:1017A000CF93DF931092CE0000E010E0C0E0D0E0D5
:1017B0000FC000E010E0C0E0D0E08091CE00E82F44
:1017C000FF27E830F10508F05EC0ED5EFF4F099499
:1017D000BEDF73D981E08093CE0082E08093CE009B
:1017E00080DF882321F08A3109F04DC004C083E0F6
:1017F0008093CE00DECF86E08093D30048C0BE0148
:1018000088279927219620919D0030919E00409134
:101810009F005091A00098DB882319F0823069F670
:1018200011C02197CE01AA27BB2721968093720071
:1018300090937300A0937400B09375000F5F1F4FD7
:1018400084E025C00115110509F0B3CF87E01CC065
:101850009ADE85E01CC0FFDD882309F0AECF83E06F
:101860008093CE0088E59BE1E6DDA7CF8091D30091
:1018700024E1829FC001112488549A4FA7D884EF95
:1018800091E053D99ACF88E08093D30086E080938B
:10189000CE0093CFA198A39AA29AA09AA998A89AA9
:1018A000AA9AAB9A80E000008F5F8A3FE1F7089523
:1018B00080E000008F5F883CE1F70895482F38E012
:1018C00090E020E8842F822311F0AA9A01C0AA9800
:1018D000AB980000999B02C0922B03C0822F809589
:1018E0009823AB9A0000315011F02695EBCFAA9ABD
:1018F000892F992708951F9310E08FEFDFDF8F3F27
:1019000011F0992705C01F5F1A30B9F78FEF90E0EB
:101910001F910895EF92FF920F931F93182F062F98
:10192000F42EE22EA8988FEFC9DF812F8064C6DFE6
:10193000802FC4DF8F2DC2DF8E2DC0DF80E0BEDFA1
:1019400085E9BCDF1F910F91FF90EF9008951F93E1
:10195000CF93DF9320E040E060E08AE0DBDFCBDF85
:10196000182F882349F4C4EDD2E08FEFA7DF8993C5
:1019700082E0C43FD807C9F7A89A8FEF9FDF812F75
:101980009927DF91CF911F9108951F93CF93DF93F4
:1019900020E040E060E089E0BDDFADDF182F882364
:1019A00049F4C4EDD2E08FEF89DF899382E0C43F30
:1019B000D807C9F7A89A8FEF81DF812F9927DF9188
:1019C000CF911F910895E1DF882329F04FEF5FEF5A
:1019D0006FEF7FEF43C08091DB028295880F880F05
:1019E000807C3091DC02232F26952695822B992727
:1019F00024E0880F991F2A95E1F7AC01662757FD6F
:101A00006095762F330F330F8091DD028295869596
:101A100086958370832B9927AA27BB27482B592BA0
:101A20006A2B7B2B4F5F5F4F6F4F7F4F8091DE02A2
:101A30008370880F2091DF02221F2227221F282B6C
:101A40008091DA028F7099270296820F911D04C04F
:101A5000440F551F661F771F8A95D2F7CB01BA0135
:101A6000089575DF982F882351F4E4EDF2E0848126
:101A7000819382E0EA3DF807D1F71092DA02892FCC
:101A800099270895AF92BF92CF92DF92EF92FF9283
:101A90000F931F93CF93DF935B016C0180916C00D8
:101AA00090916D00A0916E00B0916F008A159B051A
:101AB000AC05BD0519F480E090E05BC08FEFFEDE61
:101AC000A89820E040E060E08DE024DF14DF8FEF95
:101AD000F5DE69E0AA0CBB1CCC1CDD1C6A95D1F7B5
:101AE0008FEFECDEA89855274D2D3C2D2B2D760140
:101AF000002711276D2D7727882799274E2D81E103
:101B000009DFF9DE182F882379F58FEFD7DEC4EFD0
:101B1000D1E002C08FEFD2DE8E3F31F021978FEF00
:101B2000CF3FD807B9F702C0CD2BE9F0C4EDD0E024
:101B30008FEFC4DE899382E0C43DD807C9F78FEFE9
:101B4000BDDE8FEFBBDE8FEFB9DE8FEFB7DEA89A79
:101B50008FEFB4DEA0926C00B0926D00C0926E0068
:101B6000D0926F0004C01FEFA89A8FEFA7DE812FDD
:101B70009927DF91CF911F910F91FF90EF90DF9008
:101B8000CF90BF90AF900895CF93DF93A898B3DE26
:101B90008F3FC9F08EEF92DEC4EDD0E089918EDEEA
:101BA00082E0C43DD807D1F78FEF88DE8FEF86DE65
:101BB0008FEF84DEA0DE8F3F31F0A89A8FEF7EDEBC
:101BC00080E090E002C08FEF90E0DF91CF91089528
:101BD0001F93A89A10E08FEF71DE1F5F1A30D9F7BC
:101BE0001F9108951F93882329F020E040E060E0D2
:101BF0008CE104C020E040E060E08DE18BDE7BDE24
:101C0000182FA89A8FEF5ADE812F99271F910895D8
:101C1000CF93DF93A89A80E000008F5F883CE1F7C4
:101C200080E000008F5F883CE1F7C0E0D0E08FEFFC
:101C300045DE2196CA30D105D1F720E040E060E0D2
:101C400080E068DE58DEC7EED3E020E040E060E0F0
:101C500081E060DE50DE882331F021978FEFCF3FA7
:101C6000D80739F0F2CFA89A8FEF28DE80E090E015
:101C700005C0A89A8FEF22DE8EEF90E0DF91CF9122
:101C8000089520E030E0FC0103C02F5F3F4F319604
:101C900080818823D1F7C90108959C01FC0101C00E
:101CA000319684918823E1F7CF01821B930B08952D
:101CB000FF920F931F938C01F62EE3DF080F191F7D
:101CC000F801F08211821F910F91FF900895629F99
:101CD000D001739FF001829FE00DF11D649FE00D24
:101CE000F11D929FF00D839FF00D749FF00D659F85
:101CF000F00D9927729FB00DE11DF91F639FB00D84
:101D0000E11DF91FBD01CF0111240895AA1BBB1BC2
:101D100051E107C0AA1FBB1FA617B70710F0A61BEB
:101D2000B70B881F991F5A95A9F780959095BC010C
:061D3000CD010895FFCF74
:101D36004552524F5200FFFFFFFF1000FFFFFFFF0B
:00000001FF
